:030000000210F1FA
:03000B000200A54B
:03002B000202AE20
:03005B0002040C90
:030073000203E69F
:1000800002030406080C10182030406080040608A3
:100090000C10182030406080A0C00D0D0405060D26
:1000A0000503030302C2AFC0D0C0E020620C206889
:1000B00002419D306602415DE47385258AC262E596
:1000C00025F4700221242068022111207210758B02
:1000D00000D0E0D0D0C293C295C297D2AF32C293C3
:1000E000C295C2977406D5E0FDE53C1420E21520C8
:1000F000E10D207D02D296307D02D292020121D202
:1001000094020121207D02D292307D02D29602011A
:1001100021758B00D0E0D0D0C293C295C297D2AFE8
:1001200032758B00D0E0D0D0D2AF32419DE5256052
:100130000A207D02D293307D02D297C295419DE57F
:10014000256002D295207D02C297307D02C2934184
:100150009DE525600A207D02D297307D02D2932052
:100160007D02C293307D02C297419D207D02C292E2
:10017000307D02C296207D02C296307D02C292740A
:1001800006D5E0FDE525600A207D02D293307D0290
:10019000D297C295419D207D02C292307D02C296C7
:1001A000C2947406D5E0FDE525600A207D02D29355
:1001B000307D02D297C295419DC294207D02C292A9
:1001C000307D02C2967406D5E0FDE5256002D29529
:1001D000207D02C297307D02C293419DC294207D52
:1001E00002C296307D02C2927406D5E0FDE525601C
:1001F00002D295207D02C297307D02C293419D209C
:100200007D02C296307D02C292C2947406D5E0FD92
:10021000E525600A207D02D297307D02D293207DB1
:1002200002C293307D02C297419D207D02C296306A
:100230007D02C292207D02C292307D02C296740677
:10024000D5E0FDE525600A207D02D297307D02D2FF
:1002500093207D02C293307D02C297419D30723D52
:10026000E53C20E21A20E129207D02C292307D0285
:10027000C296207D02C296307D02C29202029D206B
:10028000E1E6207D02C292307D02C296C294020253
:100290009DC294207D02C296307D02C292E525F473
:1002A000F58A758B00D262D0E0D0D0D2AF32C2AF27
:1002B000C2AD53E6EFC0D0C0E0D2D3D2AFC2CEE5DC
:1002C0002960072074461529610C78007900E580C3
:1002D000307E01F430E30278FF53DACF207E03430F
:1002E000DA20307E0343DA10C2D8C271E580307E56
:1002F00001F430E30279FFC3E89970CE30610375F1
:1003000029182074037529188859D270E52A6004C9
:10031000152A611C20740543DA01C2D820700261DD
:1003200083A859206102C2702074367982B70431E3
:10033000C3E894F0400374F0F8E8C4540F28F87947
:1003400084B703026161C313C3138721200802C36A
:1003500013200A06C3C898F8616128F8500374FF97
:10036000F88822306915E5222408F5225003752209
:10037000FFC3E522955E4003855E227882B60418AD
:10038000852224A824C3E524955E4002A85EC3E824
:1003900095604002A8608825C3E52594404002D2BC
:1003A0006420CF0CD0E0D0D0C2D343E610D2AD321F
:1003B000C2CF7801E52960053074021529C3E559DB
:1003C00094014005755C0061DA755D00756400E5B7
:1003D0005C2401F55C5003755CFFD0E0D0D0C2D343
:1003E00043E610D2AD32C0D0C0E0C2AF53917F53CC
:1003F000E67FC260759100C3E49550F594E4955191
:10040000F595759104D0E0D0D0D2AF32C2AF53E6AB
:10041000EFC2ADC0D0C0E0C0F0D2D3D2AFA8FBA92C
:10042000FCC2D8307102817353DACF207E0343DAE5
:1004300010307E0343DA20D271E580307E01F42053
:10044000E302814A88268927C1AF53DACF207E0391
:1004500043DA20307E0343DA10C2D8C2713074020E
:10046000C19B7800E580307E01F430E302C19B88B7
:0F04700059C18253DACF207E0343DA20307E0356
:10047F0043DA10C271206102A14353DACF207E0309
:10048F0043DA10307E0343DA20C2D8D27188548900
:10049F0055C3E89552F8E99553F9E4FB7E027A00CB
:1004AF00C3E8948CE994005005755800A133C3E854
:1004BF0094C8E994005008E4D2E4FB7A0AA110C36F
:1004CF00E89468E994015008E4D2E3FB7A0FA11095
:1004DF00C3E894D0E994025008E4D2E2FB7A1EA15B
:1004EF0010C3E894A0E994055008E4D2E1FB7A3CEC
:1004FF00A110C3E89498E994085008E4D2E0FB7A7D
:10050F00787E00C3E89556FCE99557FD30E708EC77
:10051F00F42401FCEDF4FD755800C3EC9AED9E50E8
:10052F000375580188568957A854A955885289537D
:10053F007802C182C3E89526F8E99527F9307C0245
:10054F00C166307B02C166307A02C15F207502A19D
:10055F0066E9FDE8FCA185E9C313F9E813F83079E2
:10056F0002C15FE9C313F9E813F8307802C15FE9FC
:10057F00C313FDE813FC206126C3EC941CED940219
:10058F004002A19CED7018C3EC94C850120528C30B
:10059F00E528940A5002C19B755900D270C19BE5A2
:1005AF0028600215287400207F0B7888E67896B4AF
:1005BF000302789EE624FAFEE43400FFC3EC9EFCAF
:1005CF00ED9FFD92087888E6B40327A20850092012
:1005DF007D20C2AFD27DA1EE307D17C2AFC27DC2EA
:1005EF0093C295C297C292C294C296206902D26BEF
:1005FF00D2AFA2085017E6B4030DECF42401FCEDC2
:10060F00F43400FD02061C78007900C1667888E694
:10061F00B40315EC33FCED33FDC3EC940AFCED94FD
:10062F0000FD50047C007D00C3EC94FFED9400406E
:10063F000678FF7900C166EC856FF0A4C5F0A2F7CC
:10064F0033F87900400302068278FF7900020682B0
:10065F00E9C313F9E813F8307C0EE9600278FFC3A1
:10066F00E81338F8E43400F9C3E894FFE994004044
:10067F000278FF8859D270206102C19B741FF45514
:10068F002F4BF52FC274E42B7002D27475291830DA
:10069F00740375290A306102C1AF20740353DAFE67
:1006AF00752A06307403752A0AD0F0D0E0D0D0C274
:1006BF00D3D2AD43E6103279010206E47903020684
:1006CF00E4790A0206E4791E0206E479640206E47C
:1006DF0079C80206E47817E4D5E0FDD8FAD9F622F6
:1006EF007A147B7802070B7A107B8C02070B7A0D3A
:1006FF007BB402070B7A0B7BC802070BAC25752561
:10070F00017902B27DE4C294D5E0FDE5256002D205
:10071F0095D5E0FDC295D5E0FDD294D5E0FDE52558
:10072F00600A207D02D293307D02D297E570D5E02A
:10073F00FD207D02C293307D02C2977496D5E0FDF5
:10074F00D9C1EAF8D5E0FDD8FBDBB1C2948C2522E4
:10075F00C37C007D0075F00005F0EA33FAEB33FB44
:10076F0050F6EB13FBEA13FAC3E9FFE8FEE89AF839
:10077F00E99BF95004EFF9EEF8B3EC33FCED33FDE0
:10078F00D5F0DFEDF9ECF822E889F08A20D2D4F821
:10079F00A9F07B0030F70B7BFFF42401F8E9F43468
:1007AF0000F9E88520F0A4ADF0F8E98520F0A4AFBA
:1007BF00F0FEED2EF974003FFA7C04C3EA13FAE958
:1007CF0013F9E813F8DCF48BF030F70AE8F424019E
:1007DF00F8E9F43400F9E889F0C2D4F8A9F02278E6
:1007EF0082B6040302084BC3E55994014003020883
:1007FF0013852224E4F53EF53FF540F541F542F52A
:10080F004702084B7882E6FC754701E522F523780D
:10081F003879C7AA3AAB3BC3EB13FBEA13FAEC14D4
:10082F006013C3EB13FBEA13FAEC14146007C3EB6A
:10083F0013FBEA13FA12075F883E893F22E54760F0
:10084F0034C3E53E9523F8E53F9400F9500CC3E817
:10085F009480E994FF4016020880C3E8947FE994DE
:0F086F00005003020880787F79000208807880AB
:10087E0079FF8843894422E5476058E5432540F8CF
:10088E00E5443541F9854420E4300701F43542FA58
:10089E0030E709C3EA94F040150208C2C3EA940F88
:1008AE0050030208C278FF79FF7A0F0208C278005F
:1008BE0079007AF0C3E524955E5006E524600901BF
:1008CE00DBE54420E70D01DBE54430E7068840898F
:1008DE00418A4222E547700302094678A1E6FAC32F
:1008EE00E54333F8E54433F9120797E930E70BC3D4
:1008FE00E89480E994FF4013211DC3E8947FE994A6
:10090E00005002211D787F7900211D788079FFE843
:10091E0020E715C3E52398F84009C3E89401400386
:10092E000209447801020944E8F424012523F84021
:10093E000302094478FF884522E54770030209A99E
:10094E0078A2E6FAA841A942120797E930E70CC34C
:10095E00E89401E994FF4016020980C3E894FFE988
:10096E009400500302098078FF7900020980780113
:10097E0079FFE920E715C3E54598F84009C3E894E7
:10098E000140030209A778000209A7E8F424012513
:10099E0045F840030209A778FF88242278FFC26435
:1009AE00E52D5406702FD264C3E53B940A4009C36B
:1009BE00E52594405002C264E53B601974FF853B07
:1009CE00F0848537F0A4F8C5F0600278FFC3E8958F
:1009DE00615002A8618860227883E6F520120F121A
:1009EE0075E8901206C675E890E5E820ECFBA8BD08
:1009FE00A9BE120FA8756B55756C00C3740013FD5C
:100A0E00745513FC74552CFC74003DFDECFAEDFB93
:100A1E00C3E89AE99B4014E56B2455F56BE56C34FD
:100A2E0000F56CEA2CFAEB3DFB80E5AE6BAF6CC3C8
:100A3E00E56C13F9E56B13F8C3E913F9E813F8E560
:100A4E006B28F569E56C39F56A7A03C3E913F9E8A1
:100A5E0013F8DAF7AA201A7009756B00756C00028C
:100A6E000A801AEA6008EE28FEEF39FFDAF88E6B7C
:100A7E008F6C2275E890227883E6FFE5E820ECF78C
:100A8E00A8BDA9BE056DC3E56D94084052756D00F5
:100A9E00E9FA79A0E76044EA7007E56E601B020A86
:100AAE00BBC3E8956E6010E56E5006600C14020A2A
:100ABE00C70460F9020AC7E56EF56EC394A8401B21
:100ACE00755EC0C394054013755E80C39405400BDC
:100ADE00755E40C394054003755E0075BB0122EF41
:100AEE00C39401601BC3E894FFE994035012C3E85A
:100AFE00956BE9956C5009E55E601A155E020B2345
:100B0E00E55EF46010055E7888E6B40308E55E24C1
:100B1E00044002F55EA85EC3E524985002A824C3E3
:100B2E00E8955F400AA85FE55FF46003855F5E7934
:100B3E0082B70402614EC3E895604002A860882522
:100B4E00E56DB4070375BB1E22743279A387F0A43A
:100B5E00C5F0A2F733F8C3E8955E4002A85E88227E
:100B6E0088248825886122753A00753B7F2275C8D6
:100B7E0020A8CCA9CD75C824AA38AB3988388939B4
:100B8E00C3E89AF8E99BF9AA3AAB3BAC3AAD3B7E87
:100B9E00047F02C3EB940440021E1FC3EB94084073
:100BAE00021E1FC3ED13FDEC13FCDEF7C3EA9CFA25
:100BBE00EB9DFBEF6009C3E913F9E813F8DFF7EAE1
:100BCE0028FAEB39FB8A3A8B3B400122753AFF75C6
:100BDE003BFF2230600261E1854C50854D51D26061
:100BEE0043E680227892E6FFC3E535948240010FFA
:100BFE00C3E53594A040010FC3EF940640027F0574
:100C0E007E021E3072010EC3E53B940350060E0E9B
:100C1E003072010EC3E53B940250060E0E30720187
:100C2E000EA93BA83A7A04C3E913F9E813F8DAF7E8
:100C3E00C3E89EF8E99400F94009C3E89402E994E8
:100C4E000050047802E4F9E9FBE8FAC3E913FDE881
:100C5E0013FC884C894DC3EF94036037EF20E00DF1
:0F0C6E00E82CF8E93DF9ECFAEDFB020C8EE828D2
:100C7D00F8E939F9C3E89402F8E99400F97A02E445
:100C8D00FBC3EF9403400D8A4E8B4F884889498CE6
:100C9D004A8D4B22884E894F8A488B498C4A8D4B01
:100CAD002230600281AED26043E680E52D540660AD
:100CBD0027A83AA93BE53494085006E820E002A99C
:100CCD004D759100C3E498F594E499F595759104EB
:100CDD00D26053917F43E68022D265753D00752029
:100CED0000020CF9D265753D00752040E52D5406C6
:100CFD006002C265D2AF206005E53D60012278013A
:100D0D007A02C3E53B940540027802C3E53B940AA1
:100D1D0040027803C3E53B940F40027A0330690427
:100D2D00781E7A01206007E53D6003D2AF22D2AF75
:100D3D000000C2AFC3E53BFB940F40027B0FEB04F9
:100D4D003073012320620123F93069027982E58B2A
:100D5D00C39940D0053DEAFBE59E7005E59B020D6C
:100D6D0070E59A5440B52004DBEEA19D206502810B
:100D7D00F9C265759100AE3AAF3BC3E49EF594E4BC
:100D8D009FF595759104D26053917F43E68081F96B
:100D9D0030650281F9D88DD2AF2230690B05342030
:100DAD006016753400020DC520600D20650A206B9C
:100DBD0007158115810215C522A84EA94F75910001
:100DCD0053917FC3E498F594E499F5957591048555
:100DDD004850854951D26043E68022780030640541
:100DED003065027801E53575F007A4F9E5F028F5D1
:100DFD00F0E9A2F013A2F113A2F213F535C3947822
:100E0D005003753578C3E53595364008D266C293E3
:100E1D00C295C297306002C121854A50854B51D28F
:100E2D006043E68022C2AFC292C294C29630720B6A
:100E3D009001FF7406D5E0FD020E48207D02D2928E
:100E4D00307D02D296759F33759E00753C02020F60
:100E5D008DC2AF207D02C297307D02C293307217D2
:100E6D009001DCC294207D02C296307D02C2927444
:100E7D0006D5E0FD020E8790013F306206E5256044
:100E8D0002D295207D03759E23307D03759E2275BC
:100E9D003C03020F8DC2AFC292C294C29630720B48
:100EAD009001B97406D5E0FD020EB8207D02D296F0
:100EBD00307D02D292207D03759E22307D03759E7A
:100ECD0023753C04020F8DC2AFC29530721790018D
:100EDD0096207D02C292307D02C296C2947406D5D0
:100EED00E0FD020EF590012D30620EE525600A2021
:100EFD007D02D293307D02D297759F33759E00751A
:100F0D003C05020F8DC2AFC292C294C29630720BD5
:100F1D0090016B7406D5E0FD020F28D294207D035D
:100F2D00759E23307D03759E22753C06020F8DC282
:100F3D00AF207D02C293307D02C29730721F9002A6
:100F4D002A207D02C292307D02C296207D02C29679
:100F5D00307D02C2927406D5E0FD020F6D900151F5
:100F6D0030620EE525600A207D02D297307D02D2D7
:100F7D0093207D03759E22307D03759E23753C0164
:100F8D00306B13120FA87406D5E0FD7406D5E0FD85
:100F9D00D292D294D296C266D2AF2290012BC29336
:100FAD00C295C297C292C294C296C26222788076CE
:100FBD00090876090876040876010876030876FF95
:100FCD00087607087601087601087601788C760197
:100FDD000876FF0876FF0876FF0876FF0876FF088B
:100FED0076030876FF0876FF0876FF0876250876E3
:100FFD00D00876280876500876040876FF08760221
:10100D0008760008767A0876FF087601227887E65A
:10101D00FFC272BF0302D2727888E6C394036008E0
:10102D00C27DE630E102D27DC27E7889E630E102F2
:10103D00D27EC3EF94026008758E01D273021052F6
:10104D00758E00C273227880E6149000809378A18B
:10105D00F67881E6149000809378A2F6120FA822FC
:0F106D007886E61490008D9378A3F6120FA822D0
:10107C0022789CE67536FF75370CB402067536A0DF
:10108C0075370AB4030675368275370522227896B1
:10109C00E6FA7897E6FB307F047A007BFFC3EB9A85
:1010AC00FCC3948250027C82756F00056FEC856FD7
:1010BC00F0A4C3E5F0948040F222D27F119A12067C
:1010CC00D57A007B007C101206CBE5592AFA740005
:1010DC003BFBDCF37C04C3EB13FBEA13FADCF7FEFB
:1010EC00C27F119A22E5EF20E603752000052090BF
:1010FC003DFFE520146006901FFF14600093046010
:10110C000375EF12C2D353D9BF7581C043FF801250
:10111C0006C675EF0243B203E5B3240420E702F5DB
:10112C00B3120FA875800875A40075F1FF75D4F77C
:10113C0075900275A5FC75F2FC75D50075A0FD7552
:10114C00A60275F30275D60075B0FF75A70175F48C
:10115C00FF75E241120FBA1215F678988670C2AF7D
:10116C001206DF1206EF1206D51206F61206D5127B
:10117C0006FD1206D5C2AFE4F8F6D8FD78C879C8DA
:10118C00308307D9FBD8F7021C00120FBA1215F6E0
:10119C00111A1153116D117C117D1199119A7898B6
:1011AC008670120FA875885075891275C8247591B0
:1011BC000475D84075A82275B80275E690759B80A9
:1011CC00759D00759A80759C0075D10E75BC58750F
:1011DC00BB0175BA1F75E8801206C6D2AF1209E6BC
:1011EC0043DA01C2D8C2711206DF753001D2617BBD
:1011FC00037A0CE55870067A0CDB0221811206D5B5
:10120C002070022181C270E559C3940240E3E52F9E
:10121C00541F855B5AF55BB55AD7DAD7C26153DADE
:10122C00CF207E0343DA20307E0343DA10C2D8C2CB
:10123C0071C2757528001206DA307409C3E528945A
:10124C000A4002D2751206CB78023074027800C3C1
:10125C00E5599840F0C2AF1206EF1206EF1206EFF6
:10126C00D2AF1206DF7546007888E6B403026150EF
:10127C001206CB788CE6C394015003021350E53070
:10128C00C394015003021350207435C3E55994FFE5
:10129C005003021350C2AF120704D2AF1206DAC3C6
:1012AC00E559940150EFC2AF1206EF1206D01206A8
:1012BC00EFD2AF1206DAC3E55994FF40E902179E4C
:1012CC007F02D27F119A1206DAC2AFC27F119AAE98
:1012DC0059C3E559947FD2AF40741206C6C2AF12FF
:1012EC000704D2AFDFDC11C6C3EE94057897F61273
:1012FC0006DF1216381217217F0AD27F119A1206B6
:10130C00DAC2AFC27F119AAE59C3E559947FD2AFFE
:10131C0050E61206C6C2AF1206EF1206D01206EF46
:10132C00D2AFDFD611C6EE24057896F61206DF1280
:10133C0016381217501206DA119AC3E55994FF4069
:10134C00F402179EC3E5599546400385594612068B
:10135C00DA78017988E7B403027805C3E559984037
:10136C00024174C2AF120704120704120704D2AF71
:10137C001206DF753000E4F531F5320531E531F454
:10138C0070390532789AE678191460127832146044
:10139C000D787D14600878FA146003753200C3E58B
:1013AC003298401715327531B478998670C2AF12E5
:1013BC000704D2AF789886701206DA1206D0E529A7
:1013CC007005307402218178012074027806C3E51F
:1013DC00599840A77888E6C3940360031206DAE5AF
:1013EC002970022181C2AF120FA8E4F522F523F572
:1013FC0024F525D2AF78858662F53EF53FF540F5AC
:10140C0041F542F56DF547F52CF52DF535120B75BB
:10141C00756D0875BB1E1206C6120A81E5E820EC34
:10142C00FBA8BDA9BEE97001F8886E120A85756D1E
:10143C000875BB1E7887E6FE7602111A7887EEF6E1
:10144C00C2AF755EFF120B5785225E85225F852227
:10145C0060D2AF752201752401752501855D647517
:0F146C006501D268D269753400120F12120F3C5D
:10147B00120B75120B7C120BF2021492120FA811A5
:10148B001A756D0075BB01120CF1120DA7120DC66A
:10149B001207EE120DE8120E32120B7C120BE11238
:1014AB000BF2120CAE120CE6120DA7120DC612089F
:1014BB004C1209AA120DE8120E5E120B7C120BE1F4
:1014CB00120BF2120CAE120CF1120DA7120DC6126A
:1014DB000885120DE8120EA2120B7C120BE1120BF7
:1014EB00F2120CAE120CE6120DA7120DC61208E288
:1014FB00120DE8120ED4120B7C120BE1120BF2122E
:10150B000CAE120CF1120DA7120DC6120947120DDB
:10151B00E8120F12120B7C120BE1120BF2120CAE33
:10152B00120CE6120A81120DA7120DC6120A8512B1
:10153B000DE8120F3C120B7C120BE1120BF2120C8A
:10154B00AE306938206B3585615E85615F855D6482
:10155B0075650179327A0AC3E534994012C269D2B2
:10156B006A8A3385615E755FFF756020021587C3DC
:10157B00E559940140030214920215C5306A1E20EE
:10158B006B1BE533147007C26A755EFF8187F533F9
:10159B00C3E559940140030214920215C5C3E55CDF
:1015AB0094FA5016307404E529600FC3E53B78F0CC
:1015BB00306B0278609850028192C2AF120FA878FC
:1015CB0087E6FE7602111A7887EEF6E4F522F5230C
:1015DB00F524F525F562C268D2AF1206C6120FA824
:1015EB00307406E529700221816182901A0D7820F2
:1015FB0012167AE520B4550CA312167AE520B4AA7C
:10160B0003021618120FBA121638021637901A0365
:10161B0078807B0A12167AA308DBF9901A0F788C64
:10162B007B1512167AA308DBF9901A2422C2AF128B
:10163B0016B9121693901A00740D12167FA374022A
:10164B0012167FA3741312167F901A0378807B0AED
:10165B0012167EA308DBF9901A0F788C7B151216E5
:10166B007EA308DBF91216CC1216AA901A2422E4D8
:10167B0093F622E6438F01538FFD75EF0275B7A5E5
:10168B0075B7F1F0538FFE22438F02438F0175EF35
:10169B000275B7A575B7F1901A0DF0538FFC229018
:1016AB001A0D7455D17F901A0E74AAD17F227A30FD
:1016BB0079D07820901A40D17AE520F709A3DAF790
:1016CB00227A3079D0901A40E7D17F09A3DAF92238
:1016DB00AB71A872BB01027980BB02027981BB039B
:1016EB00027982BB04027984BB05027983BB0602B3
:1016FB007986BB07027992BB08027987BB0902790D
:10170B009CBB0A027988BB0B027989E8F7227C051E
:10171B001206DFDCFB22C2AF1206EF1206F6120630
:10172B00FD1207041206D01206EF1206F61206FD82
:10173B001207041206D01206EF1206F61206FD125D
:10174B000704D2AF22C2AF1207041206FD1206F62F
:10175B001206EF1206D01207041206FD1206F6123D
:10176B0006EF1206D01207041206FD1206F6120639
:10177B00EFD2AF22AE71AF72C2AF1206EF1206EF0D
:10178B001206EF1206D0DEF21207041206D0DFF8B3
:10179B00D2AF22F121F119F1197571017572017531
:1017AB007300F17F7C05AD591206DFC3ED955970BF
:1017BB00F5C3E5599401400AC3E55994FF40320241
:1017CB0017DAD1DBD138F121C2AF75EF12F119DC89
:1017DB00D50573C3E5739403500280C6F1190572E6
:1017EB00E5711490009A93F808C3E5729850028043
:1017FB00AEF1191217190571C3E571940C500280E3
:0F180B009B120FBA121638C2AF75EF12121719CF
:101A00000D02130909040103FF0701010155AA0191
:101A1000FFFFFFFFFF03FFFFFF25D0285004FF0259
:051A2000007AFF01FF48
:101A400023506C6174696E756D31353041232020EF
:101A500023424C48454C4923463331302320202033
:101A60002020202020202020202020202020202076
:101C0000C2AFC2D353D9BF7581C043B20343FF8073
:101C1000752438752503B1BF75EF0275E24043F1B5
:101C20000853A4F7D283780379E67C1075220075F7
:101C30002300901DCC7B0675249875250130830206
:101C4000813D208308D8FBD9F9DCF781AD308308CA
:101C5000D8FBD9F9DCF781ADB17FE493A3C39A60D7
:101C6000028126DBDDB171600281267B08E493FAF4
:101C7000A3B152DBF87A30B152752200752300B15E
:101C800071EAFCEBFDC3ED94FE400EB1718A278B27
:101C900028ED30E0048A828B83B1717AC270D8C398
:101CA000ED94FE601050CEBD0022EC600675200061
:101CB0000200008100A827A9280809D804D90281B8
:101CC000C9B175EA89AAF281BB0D8199C3ED94036C
:101CD0005049EDA2E092007AC5C3E5829400E58305
:101CE000941C5093200010438F02438F0175B7A5B9
:101CF00075B7F1F030001FA827A9280809438F0104
:101D0000538FFDD804D902A11689AAE275B7A5752B
:101D1000B7F1F0A3A103538FFC81757AC1BD030C09
:101D2000E493A3FAB136DCF8B12E81758177AA224B
:101D3000AB23B152EBFAEA6222752608C3E52313FE
:101D4000F523E52213F52250066323A0632201D573
:101D500026EAB1BFB1BF75260AEAF4200102D28398
:101D6000300102C283B1BFC3134002C201D526EBCA
:101D700022B175EAFB208302A175308302A17A7536
:101D80002608AE24AF25C3EF13FFEE13FEB1C3B197
:101D9000BFC3EA133083024480FA30E703632201B1
:101DA000C3E52313F523E52213F52250066323A090
:101DB000632201D526D9E52265236523F52222AECB
:101DC00024AF250E0FDEFEDFFCD20122424C486517
:0A1DD0006C6934373132F31006015C
:00000001FF
